:10000000AEC00000C7C00000C5C00000C3C00000F3
:10001000C1C00000BFC00000BDC00000BBC00000E8
:10002000B9C00000B7C0000073C40000B3C0000036
:10003000B1C00000AFC00000ADC00000ABC0000008
:10004000A9C00000A7C00000A5C00000A3C0000018
:10005000A1C000009FC000009DC000009BC0000028
:1000600099C0000097C0000095C0000093C0000038
:1000700091C000008FC000008DC000008BC0000048
:1000800089C0000087C0000085C0000083C0000058
:1000900081C000007FC000007DC000007BC0000068
:1000A00079C0000077C0000075C000001C03550037
:1000B000530042002D004D006900640069002D00CE
:1000C00032002D0043005600000016035600690060
:1000D0006B0069006E0067004300750062006500F8
:1000E00000000403090409026500020100C032098E
:1000F00004000000010100000924010001090001C1
:10010000010904010002010300000724010001416C
:100110000006240201010006240202020009240351
:100120000103010201000924030204010101000985
:1001300005010240000500000525010101090582B5
:100140000240000500000525010103120110010015
:10015000000008EB03482001000102000100112407
:100160001FBECFEFDAE0DEBFCDBF11E0A0E0B1E00F
:10017000EEE4FEE002C005900D92AA34B107D9F773
:1001800021E0AAE4B1E001C01D92A635B207E1F773
:1001900045D05BC635CF84B7877F84BF0FB6F89450
:1001A000A895809160008861809360001092600043
:1001B0000FBE90E080E80FB6F894809361009093B2
:1001C00061000FBE88D38FEF8AB91BB884B99FE056
:1001D00095B93E9A469880BB11BA6A9808954BB972
:1001E000662311F0469A01C0469845B121E030E0FF
:1001F000B90102C0660F771F8A95E2F7CB0180959F
:10020000842385B985B18F6085B908952F9A0895A3
:100210002F98089580E091E0B5C50895CF93DF93BE
:10022000CDB7DEB728970FB6F894DEBF0FBECDBFAF
:10023000B2DF78942E9A8091120190911301A091CF
:100240001401B09115018D839E83AF83B887E12C93
:10025000F12CCC24C394D12CAA24AA94BB24BA9404
:100260005FEFE51AF50A629B74C0BE016F5F7F4FB6
:1002700080E091E0C7D5882309F443C02D9A8A8194
:10028000182F1F70143009F45BC01430D0F5998119
:10029000983051F19930A9F5082F01708695817039
:1002A00032E0932E980EEB81EC53E13330F4F0E022
:1002B000E85EFE4F4081602F92DF4C8150E000905D
:1002C0000D0102C0440F551F0A94E2F7602F892DDB
:1002D00086DF123008F01E5F21B3C60101C0880F0F
:1002E0001A95EAF7822B0CC0123008F01E5F91B30A
:1002F000960101C0220F1A95EAF7822F8095892373
:1003000081BB80E091E06FD524D540E8E4164CE055
:10031000F40608F4A5CF2D98E12CF12CA1CF4FEFD6
:10032000E41AF40A629B15C0BE016F5F7F4F80E044
:1003300091E068D5811113C080E091E054D509D5D2
:10034000F0E8EF16FCE0FF0650F32D98E12CF12CBD
:10035000E6CF2F982E982D9AE0E0F8E309952D9A94
:100360008A818F70843030F4BD82BE82BF82B886AD
:1003700011BACBCF843001F78981883009F453C09A
:100380008930D1F6FE01359600E010E0CF012191D1
:100390002F3F09F041C0EB81EC53DC01A00FB11FEE
:1003A000EC930230110551F00330110561F022E0A9
:1003B000822E80E00130110521F408C093E0892EDF
:1003C00081E0912C05C083E0882E81E099249394EC
:1003D000E13330F4F0E0E85EFE4F4081692DFFDE4E
:1003E0004C8150E000900D0102C0440F551F0A944B
:1003F000E2F7692D882DF3DE902F023010F092E0A5
:10040000900F21B3A60102C0440F551F9A95E2F741
:10041000CA01822B81BB90CF0F5F1F4F04301105A3
:1004200009F0B5CF89CF2B812C53FE01359680E0A2
:1004300090E0BF013191231314C0282F823010F0B7
:1004400022E0280F31B3A60101C0440F2A95EAF734
:10045000242F2095232321BBFB01E80FF91FA08245
:100460006BCF01968430910529F766CF292F33276A
:100470002230310559F02330310569F02130310542
:10048000E9F482E190E02BE431E01CC085E690E0E5
:1004900026EE30E017C099278130910549F028F009
:1004A000029761F4ECEAF0E005C0E2EEF0E002C091
:1004B000EAECF0E0849190E09F0104C080E090E0DD
:1004C00020E030E0FA01318320830895CF92DF925B
:1004D000EF92FF920F931F93CF93DF93EC018B0169
:1004E0007A0188D1811133C0E114F10439F0F701A8
:1004F00080819181081B190BC80FD91FC12CD12CE9
:100500000115110519F18091E80085FD16C0809153
:10051000E8008B778093E8001CD4E114F10449F0E3
:10052000F70180819181C80ED91ED182C08285E0F9
:100530000EC060D1882321F30AC08091F100899315
:1005400001501109FFEFCF1ADF0ADACF80E0DF9107
:10055000CF911F910F91FF90EF90DF90CF90089572
:1005600020915401309155012617370748F0611545
:10057000710539F42091E8002E772093E80001C03E
:10058000B901FC0120E06115710571F18EB388237A
:10059000E9F18530E9F18091E80083FD3BC080916D
:1005A000E80082FD2DC08091E80080FFECCF209113
:1005B000F3008091F20090E0922B6115710551F0EB
:1005C0008830910538F421912093F1006150710930
:1005D0000196F3CF21E0089709F020E08091E80030
:1005E0008E778093E800CFCF2111D0CF09C08EB392
:1005F000882361F0853061F08091E80083FD0AC0B6
:100600008091E80082FFF3CF80E0089582E00895B2
:1006100083E0089581E008952091540130915501BF
:100620002617370748F06115710539F42091E80065
:100630002E772093E80001C0B901FC0120E061158C
:10064000710589F18EB3882309F43FC0853009F420
:100650003EC08091E80083FD3CC08091E80082FDAF
:100660002EC08091E80080FFEACF2091F3008091B6
:10067000F20090E0922B6115710559F088309105D8
:1006800040F424912093F100319661507109019654
:10069000F2CF21E0089709F020E08091E8008E7702
:1006A0008093E800CCCF2111CDCF09C08EB3882331
:1006B00061F0853061F08091E80083FD0AC080918F
:1006C000E80082FFF3CF80E0089582E0089583E0A0
:1006D000089581E00895982F973068F59093E90088
:1006E000981739F07091EC002091ED005091F000D6
:1006F00003C0242F762F50E021FD02C09F5FECCF76
:100700003091EB003E7F3093EB003091ED003D7F68
:100710003093ED003091EB0031603093EB0070933B
:10072000EC002093ED005093F0002091EE0027FDA7
:10073000E5CF80E008958F708093E90081E008950F
:100740000F931F93CF93DF93062FEC0110E0101748
:1007500071F16881611103C01F5F2596F8CF2C816C
:10076000A981BA819B81862F8F70873010F080E03D
:100770001FC0223010F442E001C046E0E8E0F0E0A3
:1007800020E0EA17FB0720F42F5FEE0FFF1FF9CFE1
:100790002295207F422B50E4959F90011124661FE3
:1007A0006627661F622B97DF8111D6CFE0CF81E0ED
:1007B000DF91CF911F910F91089580914E0187FF96
:1007C0000FC08091E80082FD04C08EB38111F9CF83
:1007D00010C08091E8008B770AC08EB3882349F05F
:1007E0008091E80080FFF9CF8091E8008E778093B8
:1007F000E80008952091E4003091E50095E64091ED
:10080000EC00842F817040FF22C08091E80080FDC1
:100810001CC08EB3882399F0853099F08091EB004D
:1008200085FD11C04091E4005091E5002417350783
:1008300031F3915011F09A01E2CF84E0089582E003
:10084000089583E0089581E0089580E0089540913F
:10085000E80042FFDECF08950F931F93CF93DF93FD
:100860004AD051D0C8EDD0E088818F7788838881C5
:100870008068888388818F7D888319BC1EBA109216
:100880004A0110924C0110924B0100EE10E0F80169
:1008900080818B7F808388818160888342E060E0F3
:1008A00080E019DFE1EEF0E080818E7F8083E2EE70
:1008B000F0E0808181608083808188608083F8019E
:1008C00080818E7F8083888180618883DF91CF9152
:1008D0001F910F910895E8EDF0E080818F7E808375
:1008E000E7EDF0E080818160808384E082BF81E079
:1008F00080934D01B1CFE8EDF0E080818E7F808361
:100900001092E20008951092DA001092E10008952A
:100910001F920F920FB60F9211242F933F934F9374
:100920005F936F937F938F939F93AF93BF93EF9357
:10093000FF938091E10082FF0AC08091E20082FF74
:1009400006C08091E1008B7F8093E10001D280910D
:10095000DA0080FF1BC08091D80080FF17C0809113
:10096000DA008E7F8093DA008091D90080FF0BC07F
:1009700080E189BD82E189BD09B400FEFDCF81E03F
:100980008EBB44DC03C019BC1EBA42DC8091E1007E
:1009900080FF17C08091E20080FF13C08091E200C9
:1009A0008E7F8093E2008091E20080618093E2007C
:1009B0008091D80080628093D80019BC85E08EBBFE
:1009C000C7D18091E10084FF2EC08091E20084FFB6
:1009D0002AC080E189BD82E189BD09B400FEFDCF56
:1009E0008091D8008F7D8093D8008091E1008F7E28
:1009F0008093E1008091E2008F7E8093E2008091FD
:100A0000E20081608093E20080914A01882311F026
:100A100084E007C08091E30087FD02C081E001C04F
:100A200083E08EBB95D18091E10083FF21C080914E
:100A3000E20083FF1DC08091E100877F8093E10089
:100A400082E08EBB10924A018091E1008E7F8093FC
:100A5000E1008091E2008E7F8093E2008091E200CD
:100A600080618093E20042E060E080E034DE70D19B
:100A7000FF91EF91BF91AF919F918F917F916F9176
:100A80005F914F913F912F910F900FBE0F901F904C
:100A900018951F93CF93DF93CDB7DEB7AA970FB604
:100AA000F894DEBF0FBECDBFEEE4F1E08091F1001F
:100AB000819321E0E635F207C9F7AFDB8091E800CA
:100AC00083FF2EC180914E0190914F01953009F422
:100AD00083C030F49130A9F168F0933091F120C1D6
:100AE000983009F4EEC0993009F4FAC0963009F054
:100AF00017C193C0803821F0823809F011C108C0B5
:100B000080914B0190914C01992389F082600FC034
:100B1000809152018F70873008F002C18093E90004
:100B20008091EB0085FB882780F91092E900909175
:100B3000E800977F9093E8008093F1001092F10015
:100B4000CBC0282F2D7F09F0EBC0882319F082300D
:100B500061F0E6C080915001813009F0E1C093302E
:100B600009F080E080934C012EC0809150018111EA
:100B70002AC0809152018F702FEF280F263008F085
:100B8000CFC08093E9002091EB0020FF1CC0933080
:100B900021F48091EB00806214C09091EB00906191
:100BA0009093EB0021E030E0A90102C0440F551FF3
:100BB0008A95E2F74093EA001092EA008091EB00F8
:100BC00088608093EB001092E9008091E800877FB5
:100BD0008093E800F2DDA4C08111A2C01091500101
:100BE0001F778091E3008078812B8093E3008091D0
:100BF000E800877F8093E800E0DD8091E80080FFD7
:100C0000FCCF8091E30080688093E300111102C063
:100C100082E001C083E08EBB83C08058823008F040
:100C20007FC080915001909151018C3D53E0950718
:100C300071F583E08A838AE289834FB7F894DE01F5
:100C4000139620E03EE051E2E32FF0E0509357008E
:100C5000E49120FF03C0E295EF703F5FEF708E2FAD
:100C600090E0EA3010F0C79601C0C0968D939D9336
:100C70002F5F243149F74FBF8091E800877F809331
:100C8000E8006AE270E0CE0101966ADC14C060916F
:100C9000520170915301AE014F5F5F4FE7DBBC0122
:100CA000892B09F43DC09091E800977F9093E8006C
:100CB00089819A81B1DC8091E8008B778093E8008C
:100CC0002FC0803869F58091E800877F8093E80025
:100CD00080914A018093F1008091E8008E7778CF6F
:100CE00081111EC080915001909151019927029766
:100CF000BCF48091E800877F8093E80080915001E8
:100D000080934A015ADD80914A01811106C0809189
:100D1000E30087FD02C081E001C084E08EBB7ADA87
:100D20008091E80083FF0AC08091E800877F80936C
:100D3000E8008091EB0080628093EB00AA960FB6EA
:100D4000F894DEBF0FBECDBFDF91CF911F91089504
:100D50000895CF938EB3882399F0C091E900CF70A6
:100D60009091EC00892F817090FD80E8C82B109243
:100D7000E9008091E80083FD8CDECF70C093E9002C
:100D8000CF910895CF93DF93EC011B8682E08C8393
:100D9000898761E0CE010196D3DC882331F061E0E0
:100DA000CE010696DF91CF91CBCC80E0DF91CF9141
:100DB00008952EB3243099F4FC0181818F708093C3
:100DC000E9002091F3008091F20090E0922B892BB2
:100DD00041F08091E8008E778093E8000BCD82E0AF
:100DE000089580E00895FC018EB3843051F4918120
:100DF0009F709093E9008091E80080FF02C0CF01CE
:100E0000D8CF08952EB3243011F080E00895FC016E
:100E100086818F708093E9008091E80082FFF5CF92
:100E20008091E80085FFF1CFCB0140E050E064E025
:100E300070E04CDB8091E80085FD05C08091E80002
:0E0E40008B778093E80081E00895F894FFCF4F
:100E4E000182400000010140000001002A01000063
:100E5E000000FFFFFFFF00380004090D11151A1ED8
:100E6E0022262B2F33373C4044494D51555A5E6252
:100E7E00666B6F73777C8084898D91959A9EA2A6FE
:0A0E8E00ABAFB3B7BCC0C4C9CD00C0
:00000001FF
